:0A00000075817F7401F58F02002E58
:10002B0002405FC294D294C2A4D2A575320075333C
:10003B000075340075350075360075370075630033
:10004B00756400754500754601754701756001754E
:10005B006101756201754800754900754A00754B61
:10006B0000754C01C233754D00755A0075590075FA
:10007B005C00755B007553007554007552F0754E3E
:10008B0000754F00755000755D00C20AC22EC20C80
:10009B00C210C211C214C215C212C213C20FC216B1
:1000AB00C217C218C219C21AC21BC21CC21DC21E61
:1000BB00C21FC220D209C234C235D236740090009E
:1000CB0030F0900031F0900032F0900033F090005F
:1000DB0034F07400900035F0900036F090027F748D
:1000EB0000F0A37404F0A37407F0A37409F090015B
:1000FB00207416F09001217401F012381012381C84
:10010B009001177401F09001227401F09001237497
:10011B0001F09001277401F09001187401F0900127
:10012B00247401F09001197401F090011A7401F01C
:10013B0090011B7401F090011F7401F090011C746D
:10014B0001F090011D7401F090011E7401F09001FB
:10015B00297401F0753C00753D0012094F7538008C
:10016B001204D912037A1204E67538001201FD123B
:10017B00403912074BC2A1120A7D120A87120A914B
:10018B00120AAF120B3D120B5B1204BF1204D912F1
:10019B0001FD1201FD753C30753D08123DA3753C08
:1001AB0000753D00123D3E123FF9121D4E121E0905
:1001BB001223E8C202C2031232281220251237D8AA
:1001CB001231B812346F122084900122E0B403066E
:1001DB001232D70201E650F8122481121C26121F8C
:1001EB00841223C90201CB783279FF0000D9FCD8E5
:1001FB00F822786479FF0000D9FCD8F82278967938
:10020B0096D9FED8FA2278FF799BD9FED8FA2278B4
:10021B000A790AD9FED8FA22E627F5270809E63724
:10022B00F528782722C3E697F5270809E697F528DE
:10023B007827228627872908098628872A1202C34E
:10024B00782C22862C08862D08862E08862F872947
:10025B0009872A1202667827792E227530007531AC
:10026B00101202A812027912029CD531F422C3E5B6
:10027B002E9529E52F952AE5309400500122E52E85
:10028B009529F52EE52F952AF52FE5309400F530BD
:10029B0022B3E52733F527E52833F52822C3E52CD0
:1002AB0033F52CE52D33F52DE52E33F52EE52F33D8
:1002BB00F52FE53033F53022E5278529F0A4F52C11
:1002CB0085F02DE528852AF0A4F52E85F02FE5285D
:0A02DB008529F0A4252DF52DE52E50
:1002E50035F0F52EE52F3400F52FE527852AF0A406
:1002F500252DF52DE52E35F0F52EE52F3400F52FBE
:1003050022E538B4101120010ED201C28174C01249
:10031500034AD282C28222E538B4200FC28174809A
:1003250012034AD282C28275380022C201A200920B
:1003350081900000E5822538F582E012034AD282D9
:10034500C282053822F954F053800F4280D282C20E
:1003550082E9C454F053800F4280221201FD22121B
:1003650001FD1201FD1201FD1201FD1201FD120137
:10037500FD1201FD22C282120360120360C281C216
:10038500831201FDD282C287C286D285D284120130
:10039500FDC282120360C281C2831201FDD282C2F4
:1003A50087C286D285D2841201FDC282120360C241
:1003B50081C2831201FDD282C287C286D285D284D0
:1003C5001201FDC282120360C281C2831201FDD2F5
:1003D50082C287C286D285C2841201FDC2821203FF
:1003E50060C281C2831201FDD282C287C286D285D4
:1003F500C2841201FDC282120360C281C28312014E
:10040500FDD282D287C286C285C2841201FDC28214
:10041500120360C281C2831201FDD282C287C286E5
:10042500C285C2841201FDC282120360C281C283E9
:100435001201FDD282D287D286D285C2841201FDF5
:10044500C282120360C281C2831201FDD282C287B9
:10045500C286C285C2841201FDC282120360C281B6
:10046500C2831201FDD282C287C286C285D284129E
:1004750001FDC282120360C281C2831201FDD282D4
:10048500C287C286C285C2841201FDC28212036080
:10049500C281C2831201FDD282C287D286D285C2B1
:1004A500841201FDC282120360D2002205A2E493E8
:1004B500A305A2F0A3DBF505A222900F1205A290D9
:1004C50000007B200204B1900F3205A29000007B52
:1004D500200204B1900F8205A29000007B20020447
:1004E500B1C283C281744012034AD282C28212020F
:1004F50011D281740012034AD282C282120211D231
:1005050081741E12034AD282C282120211D28174F0
:100515001E12034AD282C282120211D281741E12A5
:10052500034AD282C282120211D281741E12034A78
:10053500D282C282120211D281741E12034AD28261
:10054500C282120211D281741E12034AD282C28261
:10055500120211C283C281744812034AD282C28236
:10056500120211D281740412034AD282C28212028B
:1005750011D281740E12034AD282C282120211D2A2
:1005850081741512034AD282C282120211D2817479
:100595000412034AD282C282120211D28174041259
:1005A500034AD282C282120211D281740412034A12
:1005B500D282C282120211D281740412034AD282FB
:1005C500C282120211D281740012034AD282C282FF
:1005D500120211C283C281745012034AD282C282AE
:1005E500120211D281740412034AD282C28212020B
:1005F50011D281740412034AD282C282120211D22C
:1006050081740412034AD282C282120211D2817409
:100615000412034AD282C282120211D281741512C7
:10062500034AD282C282120211D281740E12034A87
:10063500D282C282120211D281740412034AD2827A
:10064500C282120211D281740012034AD282C2827E
:0E065500120211C283C281745812034AD2826B
:10066300C282120211D281740412034AD282C2825C
:10067300120211D281740E12034AD282C282120272
:1006830011D281741512034AD282C282120211D28C
:1006930081740412034AD282C282120211D281747B
:1006A3001512034AD282C282120211D281740E122F
:1006B300034AD282C282120211D281740412034A03
:1006C300D282C282120211D281740012034AD282F0
:1006D300C282120211222430F02275F00A84AFF094
:1006E30075F00A84E5F02430F0EF2430A3F022758E
:1006F300F00A84AFF075F00A842430F0E5F024307A
:10070300A3F0EF2430A3F0221206F2A3742CF0EE30
:100713002430A3F022D281C2831201FDD282D28778
:10072300D286D285D2841201FDC282120360D281A5
:10073300C2831201FDD282D287D286D285D284129D
:1007430001FDC282120360221204D91201FD1201BB
:10075300FD1201FD1201FD1201FD1201FD1201FD49
:100763001204BF753C24753D001201FD1201FD7595
:100773003C30753D001201FD1201FD753C20753DB5
:10078300021201FD1201FD753C20753D081201FDA9
:100793001201FD753C20753D201201FD1201FD750E
:1007A3003C20753D801201FD1201FD753C20753D15
:1007B300101201FD1201FD753C20753D041201FD6F
:1007C3001201FD753CA0753D001201FD1201FD757E
:1007D3003C60753D001201FD1201FD753C28753D1D
:1007E300001201FD1201FD753C22753D001201FD51
:1007F3001201FD753C20753D001201FD1201FD75CE
:100803003C20753D001201FD1201FD753C20753D34
:10081300401201FD1201FD753C21753D001201FDE1
:100823001201FD753C20753D011201FD1201FD759C
:100833003C20753D001204CC1201FD1201FD120192
:10084300FD1201FD1201FD1201FD1201FD1201FD58
:100853001201FD1201FD1201FD1201FD1201FD1233
:1008630001FD1201FD1201FD1201FD1201FD120134
:10087300FD1201FD1204D91201FD1201FD1201FD49
:100883001201FD221201FD1201FD1201FD1201FDF3
:100893001201FD1201FD1201FD1201FD1201FD12F3
:1008A30001FD1201FD1201FD1201FD1201FD1201F4
:1008B300FD1201FD1201FD1201FD1201FD1201FDE8
:1008C3001201FD1201FD1201FD1201FD1201FD12C3
:1008D30001FD1201FD1201FD1201FD1201FD1201C4
:1008E300FD1201FD1201FD1201FD1201FD1201FDB8
:1008F3001201FD1201FD1201FD1201FD2220B204BD
:100903007539002220B103D2042275390122E53959
:10091300B53A0485393A22B4001920040A053B8507
:10092300393AD206D20222153BC20485393AD2069D
:10093300D2032220040A153B85393AD206D2032278
:10094300053BC20485393AD206D20222C2B3C2B4ED
:10095300C2B5E53CF4200E0244FE7F083392B6D2C2
:10096300B5C2B5DFF7B2B30000C2B3E53DF4200E64
:100973000244FE79083392B6C2B5D2B5D9F7D2B4E0
:100983000000C2B422C293D2937908C290A29133D9
:10099300D290D9F7F53EC293D2937908C290A2922E
:1009A30033D290D9F7F53F22E582C4540FF9E5839A
:1009B300C46922E5820303543FF9E583030354C06A
:1009C30069227A0CC2A6D2A3A2C133C933C9C2A376
:0E09D300DAF2F8D2A622C2A3C2A63392A7D2AD
:1009E100A3DAF5C2A31209C5E95403F9227A057401
:1009F100C01209D9F5838882227A0574C81209D9EF
:100A0100F5838882227A0574D01209D9F583888208
:100A1100227A0574D81209D9F58388822285823217
:100A210085833375340075350078327536787537BE
:100A310000793612023E8552367537037936120235
:100A41004EE6228582328583337534007535007810
:100A510032753611753700793612024EE62222C2FE
:100A6100A0E8120A71E9120A71EA120A71D2A022EF
:100A71007B08D2A13392A2C2A1DBF7227840790F81
:100A81007A00120A60227869790F7A00120A6022CC
:100A9100787779007A00120A6022782F79FF7AF04C
:100AA100120A6022782F79807A00120A6022782F48
:100AB10079007A00120A6022782FF97A00120A600E
:100AC10022782F791F7A80120A6022782F793F7A53
:100AD10000120A6022782F79FC7A00120A6022E55E
:100AE10083C454F0F9E582C4FA540F49F9EA54F089
:100AF100FA22120AE07800120A6022120AE0780152
:100B0100120A6022120AE07802120A6022120AE036
:100B11007803120A6022120AE078A0120B2022C286
:100B210096E8120B31E9120B31EA120B31D29622FF
:100B31007B08D2A1339295C2A1DBF72278277900F5
:100B41007A00120B202278A079FF7AF0120B202272
:100B510078A079807A00120B202278A079007A009F
:100B6100120B202278A0791F7A80120B202278A004
:100B7100793F7A00120B202278A079FC7A00120BBF
:100B81002022F532753300783275362275370079B7
:100B91003612023E868208868322F532753300784A
:100BA10032753622753700793612023E8682088602
:100BB1008322120E44F532753300783275362A7568
:100BC1003700793612023E868208868322F5327515
:100BD10033007832753620753700793612023E8639
:100BE1008208868322900030E004B410027400F081
:100BF100900020A98229F582E022900034E0FA9049
:100C01000031E004B40F0274FFF0900EF2932A90C9
:100C11000034F0900033E004B410027400F0F99055
:100C21000034E0FA900020E58229F582EAF0229072
:100C31000034E0FA900032E004B4110274FFF09045
:100C41000F01932A900034F0120C1422120BE65477
:100C5100016008120BE6541F246022747F22F9748C
:100C6100FF89F084F5F0120BE68422120BE675F091
:100C7100208422120BE675F03384240122120BE644
:100C810075F02084240122120BE675F03F842401C3
:100C910022120BE675F03384240322120BE675F061
:100CA100108422120BE675F01F8422120BE675F0F8
:100CB1002084F8120BE675F03F842822120BE654CB
:100CC1000175F00CA422120BE675F0558475F00C39
:100CD100A422B40101225003740122B4070122505D
:100CE1000122740722B40101225003740122B40AC3
:100CF1000122500122740A22B4010122500374011D
:100D010022B40D0122500122740D22B4010122509E
:100D110003740122B4100122500122741022B40183
:100D210001225003740422B40401225001227401EF
:100D310022B40101225003740A22B40A0122500193
:100D410022740122B40101225003741822B4180143
:0E0D510022500122740122B4010122500374C9
:100D5F000122B43A0122500122743A22B401012235
:100D6F005003740122B4460122500122744622B46A
:100D7F000101225003740122B40401225001227494
:100D8F000422B40101225003740122B40501225040
:100D9F000122740522B40101225003740122B420F0
:100DAF000122500122742022B40101225003740148
:100DBF0022B4020122500122740222B401012250F6
:100DCF0003740122B4020122500122740222B401E1
:100DDF0001225003740122B405012250012274052F
:100DEF0022B40001225003740022B40501225001E5
:100DFF0022740522B40001225003740022B40301AF
:100E0F0022500122740322B4FF03740C22B40B018D
:100E1F0022500122740C22B4FF02EC22B43C0122B6
:100E2F00500122EC22B4FF03740022B403012250BC
:100E3F000122740322B46001224002746022B4FFC5
:100E4F0003740022B4240122500122742422B4011D
:100E5F0001225003740122B4180122500122741888
:100E6F0022B40101225003740122B4020122500165
:100E7F0022740222B40101225003740122B4020130
:100E8F0022500122740222F990027AE0F55EE9B451
:100E9F000101225003740122B55E0122500122E5A7
:100EAF005E22F990027AE0F55EE9B4010122500367
:100EBF00740122B55E0122500122740122B4010196
:100ECF00225003740422B40401225001227401221F
:100EDF00B40101225003740122B40C0122500122EB
:100EEF00740C22037F2C0C0105712133E6FF0B5785
:100EFF006818BD09A60D004B5D263585B1961140CA
:100F0F0093C8D3204620204C20204120204D202064
:100F1F0045202043484F5244204D414348494E45B8
:100F2F00203220202056455253494F4E20312E302B
:100F3F003020202020286329323031362D323031B5
:100F4F00372020496E697420616C6C204461746194
:100F5F00203F204F4B202020202020202020202009
:100F6F004E4F2020506C6561736520776169742046
:100F7F002120202020202020202020202020202061
:100F8F002020202020202020202020202020202052
:100F9F002020204D4F44452050524F4752414D4D38
:100FAF002020204D4F44453C3E20234330202052EB
:100FBF004F4F542020503031202023433120202008
:100FCF002020202020503031204449523A646F773E
:100FDF006E204449563A6E6F20202343312001730F
:100FEF0063616C653A503031202023433120027306
:100FFF0063616C653A5030312020234331200373F5
:10100F0063616C653A50303120202043484F524481
:10101F0020204152502F514152504547494F2020D7
:10102F005155414E54204C454E4748542053454C42
:10103F004543544C6973743A413031202020434862
:10104F004F52444C6973743A413031202020415241
:10105F00502F51202041322020553031203C20325A
:10106F006E643E3C63686F7264204172706567679F
:10107F00696F3E3C7363616C652041727065676791
:10108F00696F3E3C737461626C2E5175616E746949
:10109F007A653E3C636C6F636B205175616E74694A
:1010AF007A653E63686F72647363616C65207570F7
:1010BF0020646F776E616C7431616C743272616E23
:0E10CF00646E6F202020646972656374207067
:1010DD00657220435620202020737465702062793C
:1010ED0020737465706F6666206F6E43484F52446F
:1010FD0020202020205343414C4520202020204BF0
:10110D0045594E4F54453A20204C4953543A41309D
:10111D00312020534554555020202020204152503D
:10112D00454747494F202053415645202020202038
:10113D0020726F6F7420203173742020326E642002
:10114D0020337468205452414E53504F53453A202A
:10115D0020494E505554202020204F6374617665F0
:10116D002052616E67654F637461766520547261BC
:10117D006E73706F736520312D4F637420446972E7
:10118D00656374696F6E20322D4F637420446972EC
:10119D00656374696F6E20332D4F637420446972DB
:1011AD00656374696F6E20202053455454494E4732
:1011BD005343484F5244203E205530315343414C08
:1011CD0045203E205530312020204C495354203E9F
:1011DD0020415072657373206B65792043484F52DF
:1011ED004421202053544F52414745204F4B20213D
:1011FD0020202054554E452D4D4F4445202041551E
:10120D00544F4C4F4144206C61737420736176656B
:10121D0064204C6973742020202020202020204C35
:10122D006973743A20415365742043562D4F5554BC
:10123D00733A202B38564B45594E4F54453A202082
:10124D00432343204423442045204623462047235F
:10125D0047204123412042030000000004000C0000
:10126D000C03000C180C04000C18240200070007D6
:10127D000400070E1502000500050400050A0F0203
:10128D0000040004030004080C0200030003030023
:10129D0003060C040003070E0400030A11040003E7
:1012AD00060A0400030A0E040003070B03000306DD
:1012BD000C040003070A0400030709030003070CCD
:1012CD00030004070C0400040709040004070A04C2
:1012DD000004070B030005070C030002070C0400B4
:1012ED0004090E030004080C030004060C04000599
:1012FD00070A040004080A040004060A0400040B8B
:10130D000E0400040B0D0400040B0F040004070E63
:10131D0004000B0E1104000B101504000B0E150428
:10132D0000040B12030000000020202020202020AC
:10133D002020554E49534F4E4F2020202020202055
:10134D004F4354415645532031202020202020204A
:10135D004F43544156455320322020202020202039
:10136D004F43544156455320332020202020202028
:10137D00202046494654482031202020202020207E
:10138D00202046494654482032202020202020206D
:10139D0020464F5552544820312020202020202017
:1013AD0020464F55525448203220202020205448AA
:1013BD00495244206D616A203120202020202020B8
:1013CD004155474D454E544544202020202054483A
:1013DD00495244206D696E20312020202020204468
:1013ED00494D494E495348454420202020204D4920
:1013FD004E4F522061646420392020202020204D42
:10140D00494E4F5220372F31312020202020204DA2
:10141D00494E4F5220372062352020202020202099
:10142D004D494E4F5220372F3920202020204D4935
:10143D004E4F52206D616A20372020202020202021
:0E144D00204D494E4F52206235202020202095
:10145B00202020204D494E4F522037202020202085
:10146B00202020204D494E4F522036202020202076
:10147B002020202020204D494E4F5220202020207C
:10148B002020202020204D414A4F52202020202078
:10149B00202020204D414A4F522036202020202052
:1014AB00202020204D414A4F522037202020202041
:1014BB004D414A4F52206D616A2037202020202059
:1014CB004D414A4F52207375732034202020202029
:1014DB004D414A4F5220737573203220202020201B
:1014EB0020204D414A4F5220362F392020202020DA
:1014FB002020204D414A4F522023352020202020F0
:10150B002020204D414A4F522062352020202020A0
:10151B0020204D414A4F5220372F342020202020AD
:10152B00204D414A4F5220372023352020202020A8
:10153B00204D414A4F522037206235202020202059
:10154B0020204D414A4F5220372F39202020202078
:10155B00204D414A4F522037206239202020202035
:10156B00204D414A4F522037202339202020202064
:10157B004D414A4F52206164642039202020204D78
:10158B00414A4F5220372F392F3131202020202034
:10159B00204D414A4F5220372F3133202020204DF0
:1015AB00414A4F5220372F392F3133202020202012
:1015BB004D414A4F522037622031312020202020CC
:1015CB0020202020554E49534F4E4F2020202020C5
:1015DB0020757365722063686F72640800020305DF
:1015EB000607080B000000000600010405070800B1
:1015FB0000000000000500010307080000000000C8
:10160B0000000600030407090A00000000000006A2
:10161B0000030506070A0000000000000700010494
:10162B000507080B00000000000C00010203040575
:10163B00060708090A0B0500020407090000000051
:10164B00000000070001040507080B000000000064
:10165B000700010406080A0B000000000005000249
:10166B0005070A0000000000000007000204050740
:10167B00080A0000000000070003040607090A001F
:10168B0000000000070002030607080B0000000023
:10169B000005000203070800000000000000050021
:1016AB000105060A00000000000000050001050707
:1016BB00080000000000000005000105070A0000FB
:1016CB00000000000005000305070A0000000000F1
:1016DB00000005000205070A0000000000000005DD
:1016EB0000020407090000000000000007000204CC
:1016FB000506080A000000000007000103040608A5
:10170B000A0000000000070002040607080A000098
:10171B00000000070002030507080B000000000093
:10172B00070001030506090A00000000000700027C
:10173B00040508090B000000000007000203060760
:10174B00090A0000000000070001040507080A0051
:10175B0000000000070003040607090B000000004F
:10176B000007000103040608090000000000070041
:10177B0002030507090B0000000000070002040527
:10178B0007090B0000000000070002030507090A08
:10179B000000000000070001030507080A00000015
:1017AB000000070002040607090B000000000007F9
:1017BB000002040507090A000000000007000203ED
:0E17CB000507080A00000000000700010305E2
:1017D90006080A0000000000070001030507090BBD
:1017E9000000000000070001030507080B000000C6
:1017F90000000900020304060708090B000000089D
:10180900000103040607090A00000000070001049B
:101819000506090A0000000000070002040607097E
:101829000A0000000000050001030708000000008D
:101839000000000500020507090000000000000083
:10184900050002040709000000000000000500036C
:1018590005070A0000000000000005000204060A4E
:1018690000000000000000070001040507080A0045
:101879000000000008000103040607090A0000002F
:10188900000600020406080A000000000000070024
:10189900020406080A0B0000000000202020202076
:1018A900202020416C67657269616E20202020200C
:1018B900202020204172616269616E202020202051
:1018C9002042616C696E657369616E202020202059
:1018D900426C756573206D616A6F7220202020202B
:1018E900426C756573206D696E6F7220202020200F
:1018F900202042797A616E74696E6520202020204B
:1019090020204368726F6D61746963202020202054
:10191900202020446961746F6E696320446F756289
:101929006C65204861726D6F6E69632020202020EC
:101939002020456E69676D6174696320202020202D
:10194900202020456779707469616E20202020204D
:10195900202048696E64757374616E2048756E67DE
:10196900617269616E206D616A6F722048756E6778
:10197900617269616E206D696E6F724A6170616E24
:101989003A2068697261796F7368694A6170616E3A
:101999003A697761746F796F7368694A6170616ECA
:1019A9003A6B756D6F69796F7368694A6170616EB9
:1019B9003A2020202020696E73656E4A6170616E3D
:1019C9003A2020202020796F73656E4A6170616E1C
:1019D9003A2020726974737573656E4A6170616E1D
:1019E9003A2020202072796F73656E2020206D6166
:1019F9006A6F72204C6F637269616E202020737563
:101A0900706572204C6F637269616E202020204CD2
:101A1900796469616E206D696E6F724D696E6F725E
:101A2900206861726D6F6E696320314D696E6F72E6
:101A3900206861726D6F6E696320324D696E6F72D5
:101A4900206861726D6F6E696320334D696E6F72C4
:101A5900206861726D6F6E696320344D696E6F72B3
:101A6900206861726D6F6E696320354D696E6F72A2
:101A7900206861726D6F6E696320364D696E6F7291
:101A8900206861726D6F6E696320372020204D696F
:101A99006E6F72206D656C6F6469634D6F64653A32
:101AA90020496F6E69616E2F4D616A4D6F64653AA9
:101AB9002020202020446F7269616E4D6F64653A61
:101AC900202020506872796769616E4D6F64653AAC
:101AD90020202020204C796469616E4D6F64653A3D
:101AE900204D69786F6C796469616E4D6F64653AF0
:101AF90041656F6C69616E2F4D696E4D6F64653A12
:101B0900202020204C6F637269616E4E6561706F91
:101B19006C6974616E206D616A6F724E6561706F78
:101B29006C6974616E206D696E6F722020202020AF
:101B390020204E696E6520546F6E6520202020207C
:0E1B490020204F637461746F6E69632020204A
:101B570020202020204F7269656E74616C20202040
:101B670020202020204F766572746F6E652020201C
:101B7700202020202020202050656C6F6720202007
:101B870020202050656E7461746F6E69636D616AA1
:101B97006F722050656E7461746F6E69636D696EE4
:101BA7006F722050656E7461746F6E6963202020B8
:101BB70020202050726F6D65746865757320202032
:101BC7002020202020205370616E69736820202018
:101BD700202053796D6D6574726963616C202020D4
:101BE7002020202057686F6C65746F6E656C656187
:101BF70064696E6757686F6C65746F6E6520202027
:101C070020202075736572207363616C6501000085
:101C1700000001000000000000000000000000E5D7
:101C27003F30E407121C63121D9622121C39121C46
:101C37004E2220020122C205900117E004120CD3A4
:101C4700F0121CABC2022220030122C20590011729
:101C5700E014120CD3F0C203121CAB22E53E30E1B4
:101C67000122E53E30E01530E31730E52DE53F3042
:101C7700E72330E11130E21830E310227401021C2F
:101C8700A37402021CA37403021CA37404021CA302
:101C97007405021CA37406021CA37407900117F0B5
:101CA700121CAB22900117E01475F003A4901CB826
:101CB70073021CCD021CDD021CED021CFF021D1865
:101CC700021D2B021D387401900117F0121D4E12D0
:101CD70020251237D8227402900117F0121D4E12D8
:101CE70024671237F4227403900117F0121D4EE592
:101CF7004E1234921234FE227404900117F0121D12
:101D07004E12291C533C21533D41433C14433D286B
:101D1700227405900117F0121D4E533C21533D418B
:101D2700433D28227406900117F0121D4E1227FA20
:101D3700227407900117F0121D4E533C21533D4169
:101D4700433C02433D2822900117E0B4010690105E
:101D5700F8021D8BB40206901102021D8BB4030614
:101D670090110C021D8BB40406901116021D8BB442
:101D77000506901120021D8BB4060690112A021D3C
:101D87008B90113405A29000007B0A1204B12290B7
:101D97000117E01475F003A4901DA373021DC6027A
:101DA70021DE02337C02284B0239E00227C50238C4
:101DB70028900F8205A29000097B041204B1221219
:101DC7001DD9121DF1121E091221151235F31235F4
:101DD700932220020122C205900120E004120D582F
:101DE700F0900120F0C202D2342220030122C20562
:101DF700900120E014120D58F0900120F0C203D298
:101E07003422900120121E16900120121F6A22E030
:101E1700B42B069015D6021F5650F81475F006A479
:101E2700901E2B73901336021F24901346021F2413
:101E3700901356021F24901366021F2490137602F4
:101E47001F24901386021F24901396021F249013B9
:101E5700A6021F249013B6021F249013C6021F2444
:101E67009013D6021F249013E6021F249013F60244
:101E77001F24901406021F24901416021F24901486
:101E870026021F24901436021F24901446021F2492
:101E9700901456021F24901466021F249014760291
:101EA7001F24901486021F24901496021F24901456
:101EB700A6021F249014B6021F249014C6021F24E2
:0E1EC7009014D6021F249014E6021F249014DB
:101ED500F6021F24901506021F24901516021F24D2
:101EE500901526021F24901536021F2490154602D0
:101EF5001F24901556021F24901566021F24901565
:101F050076021F24901586021F24901596021F2421
:101F15009015A6021F249015B6021F249015C6051C
:101F2500A29000107B101204B112216990000D746B
:101F350050F02205A29000107B101204B1900F8280
:101F450005A290000A7B031204B190000D7450F0B5
:101F55002205A29000107B101204B1122169900095
:101F65000D7455F022E0B42B03021F7A50FB90004C
:101F75000E1206DD22C3942A90000E1206DD2220E1
:101F8500340122C234121FA61221A31220251237B2
:101F9500D8900120E0F56990015A123B85E569F07A
:101FA50022900120E0B42B03021FEF50FB1475F0C3
:101FB50005A4FB90126493FC0BEB93254EFD0BEBF4
:101FC50093254EFE0BEB93254EFF0BEB93254E9081
:101FD500003CF090003BEFF090003AEEF0900039B5
:101FE500EDF0900038ECF0F56022123D5590027F3F
:101FF500E0FBA3E0254EFCA3E0254EFDA3E0254E26
:10200500FEA3E0254E90003CF090003BEEF09000E2
:102015003AEDF0900039ECF0900038EBF0F56022E5
:10202500533C21533D41E560B4000122B4010890C1
:102035000039E01220CC22B4020F900039E01220C2
:10204500CC90003AE01220CC22B40316900039E07F
:102055001220CC90003AE01220CC90003BE01220F8
:10206500CC22900039E01220CC90003AE01220CC2E
:1020750090003BE01220CC90003CE01220CC229056
:102085000117E0B40507300C04123AEF229000392D
:10209500E025532555120BB3120AF390003AE025BB
:1020A500532555120BB3120AFC90003BE02553252E
:1020B50055120BB3120B0590003CE0255325551224
:1020C5000BB3120B0E2222F9E56375F00CA4C3C9FC
:1020D50099120E1675F004A49020E173433C022278
:1020E500433C0422433C0822433C1022433C40220B
:1020F500433C8022433D0222433D0422433D0822C6
:10210500433D1022433D2022433D8022433D002292
:10211500900117E0B4010302212022E53E30E101E0
:1021250022E53E30E20AE53F30E01FC210C211222F
:10213500201016D210900142123B85E004120D1FAB
:10214500F0900124F01221962222201116D211902E
:102155000142123B85E014120D1FF0900124F0128C
:1021650021962222900124E01475F006A490217690
:102175007390113E02218B90114302218B901148DF
:1021850002218B90114D05A29000087B051204B128
:1021950022121FA61221A31220251237D822900140
:1021A50024E0B4010122B40208900039E0240CF0C7
:1021B50022B4030F900039E0240CF090003AE0249B
:1021C5000CF022900039E0240CF090003AE0240C49
:1021D500F090003BE0240CF0221221FB1222131296
:1021E500222B900F8205A29000087B051204B112E4
:1021F50035F31235932220020122C205900121E018
:1022050004120D6BF0900121F0C202D23522200399
:102215000122C205900121E014120D6BF0900121FD
:10222500F0C203D2352290012112223B121DB89033
:1022350001211223AF22E0B43707901C04121F5668
:0E2245002250F7B42B03022250400BC3942BFF
:1022530075F006A4902360731475F006A4902264AD
:10226300739018A40223AB9018B40223AB9018C444
:102273000223AB9018D40223AB9018E40223AB9053
:1022830018F40223AB9019040223AB901914022310
:10229300AB9019240223AB9019340223AB90194459
:1022A3000223AB9019540223AB9019640223AB9021
:1022B30019740223AB9019840223AB90199402235F
:1022C300AB9019A40223AB9019B40223AB9019C4A9
:1022D3000223AB9019D40223AB9019E40223AB90F1
:1022E30019F40223AB901A040223AB901A140223AD
:1022F300AB901A240223AB901A340223AB901A44F6
:102303000223AB901A540223AB901A640223AB90BE
:102313001A740223AB901A840223AB901A940223FB
:10232300AB901AA40223AB901AB40223AB901AC445
:102333000223AB901AD40223AB901AE40223AB908E
:102343001AF40223AB901B040223AB901B14022349
:10235300AB901B240223AB901B340223AB901B4492
:102363000223AB901B540223AB901B640223AB905C
:102373001B740223AB901B840223AB901B94022398
:10238300AB901BA40223AB901BB40223AB901BC4E2
:102393000223AB901BD40223AB901BE40223AB902C
:1023A3001BF40223AB901C04121F3822E0B4370342
:1023B3000223BF50FB90000E1206DD22C394369019
:1023C300000E1206DD2220350122C2351223E81247
:1023D30024671237F4900121E0F5699001A2123BC2
:1023E30085E569F022900121E0B4370A123D6F9030
:1023F300003DE0F5612250F412243905A290003D1E
:10240300F0F56112242822B4370A123D8990004A5C
:10241300E0F5622250F412243905A290004AF0F547
:102423006212242822A305A20BEB9305A2254EF0EA
:10243300A305A2DAF322B413030224415006901534
:10244300E602245EB4260302244F50099016DDC32E
:10245300941302245E9017D4C394261475F00DA42C
:10246300FB93FA22533C21533D4190003DE0FA7027
:102473000122A3E005A21220CC05A2DAF522120A5A
:10248300121209B6B4370302249A500BD294533C68
:10249300FE533DFEC20922433C0130090122D20909
:1024A3001546E54660012212274F12252A9001EABC
:1024B300123B85E0F546C294433D01E545B5470926
:1024C3007545001232C70224CE50F51224F61224A9
:1024D300D7054522E02553254925561224E222F942
:1024E300900117E0B40504300C0122E9120BB3127A
:1024F3000B1722E54CB405041225132212250322DF
:102503009000B7E5822545F582E5833400F5832203
:10251300E547120C5FF5459000B7E5822545F58246
:10252300E5833400F58322900172123B85E0B40108
:102533000412253F22B4020312256A22E54CB4019A
:10254300079000B71225B022B402079000B71225F6
:10255300E022B4030412264722B4040412265E22A6
:102563009000B71225B022E54CB401079000B712D2
:10257300268D22B402079000B71226BD22B40304AD
:1025830012272422B4040412273B229000B71226F8
:102593008D22E56070057E01790122FEF922E56056
:1025A300B402057E0279022240F9FEF92212259532
:1025B300AB4B0B7A0005A29000391225D4EEF9EA51
:0E25C300240CFA900039DBF2E54B048EF0A4F4
:1025D100F54722E02AA305A2F0A305A2D9F522120C
:1025E1002595AB4BEB75F00CA4FA0B05A2900038C6
:1025F100123BB612260FEEF9EAC3940CFA9000389A
:10260100123BB6DBEEE54B048EF0A4F54722E02A3F
:10261100FF123BA805A2EFF0A305A2D9F1221225D2
:10262100A119AB4BEB75F00CA4FA0B05A290003885
:10263100123BB612260FEEF9EAC3940CFA90003859
:10264100123BB6DBEE229000B71225B005A212268E
:102651001FE54775F002A4C39402F547229000B725
:102661001225B005A21225E0E54775F002A4F54751
:1026710022E56170057E01790122FEF922E561B44E
:1026810002057E0279022240F9FEF922122672AB7E
:102691004B0B7A0005A290003E1226B1EEF9EA2416
:1026A1000CFA90003EDBF2E54B048EF0A4F54722D4
:1026B100E02AA305A2F0A305A2D9F522122672AB46
:1026C1004BEB75F00CA4FA0B05A290003D123BB642
:1026D1001226ECEEF9EAC3940CFA90003D123BB6D7
:1026E100DBEEE54B048EF0A4F54722E02AFF123B16
:1026F100A805A2EFF0A305A2D9F12212267E19ABFB
:102701004BEB75F00CA4FA0B05A290003D123BB601
:102711001226ECEEF9EAC3940CFA90003D123BB696
:10272100DBEE229000B712268D05A21226FCE547AA
:1027310075F002A4C39402F547229000B712268DCA
:1027410005A21226BDE54775F002A4F5472212271E
:10275100B8900127E0B401149001D2123B85E0F555
:102761004CE54A120E03F54B75490022B40218904C
:1027710001D2123B85E0F54C754B00E54A120DF094
:1027810075F00CA4F54922B4030EE54A120D91F53A
:102791004C754B0075490022B4040EE54A120D91A7
:1027A100F54C754B0175490022E54A120D91F54C26
:1027B100754B0275490022120A06120A1E75F00CA9
:1027C10084F54A221227CC1227E32220020122900B
:1027D1000127E004120DDDF0900127F01227FAC263
:1027E100022220030122900127E014120DDDF09056
:1027F1000127F01227FAC20322533C21533D419095
:10280100115C05A29000097B071204B11228112264
:10281100900127E0120DDDF01475F006A490282236
:102821007390116302284090117302284090118324
:102831000228409011930228409011A302284005DC
:10284100A29000107B101204B1221228E312285822
:10285100122E0A12359322E53E30E1041228A422F9
:1028610012286522E53E30E222E53F30E005C21044
:10287100C21122201014D210900129E004120EDF9F
:10288100F0123FEE12291C12322822201114D2110B
:10289100900129E014120EDFF0123FEE12291C12F2
:1028A100322822E53E30E222E53F30E005C210C287
:1028B1001122201014D21090011AE004120D45F0DB
:1028C100122AF912291C12322822201114D2119035
:1028D100011AE014120D45F0122AF912291C1232C4
:1028E1002822E53E20E10122E53F30E60AE53E30BF
:1028F100E417C214C2152220140ED214900119E05B
:1029010014120D32F012291C2220150ED21590013D
:1029110019E004120D32F012291C22900119E0B4C1
:102921000124122B10900FB605A29000107B01120A
:1029310004B190012A122C61900FB705A2900014E6
:0E2941007B011204B122B40221122B10900F60
:10294F00B605A29000157B011204B1122C92900FC4
:10295F00B705A290001A7B011204B122B40328120A
:10296F002B10900FB605A290001B7B011204B190A3
:10297F00015A123B85E0122CC2900FB705A29000AE
:10298F001F7B011204B122B40404122B4422B40998
:10299F0004122B5B22B40A04122B9922900172129B
:1029AF003B85E0B40304122A562250FA1229BF22A3
:1029BF00900119E0B40527122BB0900FB605A29025
:1029CF0000107B011204B190018A122C81900FB775
:1029DF0005A29000147B011204B1122D9322B406AC
:1029EF0021122BB0900FB605A290001B7B01120491
:1029FF00B1122D93900FB705A290001F7B01120407
:102A0F00B122B40721122BDA900FB605A290001352
:102A1F007B011204B1122DB5900FB705A2900018CB
:102A2F007B011204B122122BDA900FB605A290008F
:102A3F001C7B011204B1900FB705A290001F7B0100
:102A4F001204B1122DEB22900119E0B40524122CBF
:102A5F0001900FB605A29000107B011204B19002F5
:102A6F0002122C81900FB705A29000147B01120463
:102A7F00B122B40627122C01900FB605A290001BAD
:102A8F007B011204B1900232123B85122CE8900F99
:102A9F00B705A290001F7B011204B122B4072412C4
:102AAF002C31900FB605A29000107B011204B1904B
:102ABF00021A122C81900FB705A29000147B0112FD
:102ACF0004B122122C31900FB605A290001B7B018E
:102ADF001204B190024A123B85122CE8900FB705F1
:102AEF00A290001F7B011204B12290011AE0900006
:102AFF00061206DD22900129E0142441900005F012
:102B0F0022122B04122AF990101805A29000097BAB
:102B1F00071204B1900FB805A29000107B10120499
:102B2F00B190012A122C61122C9290015A123B85FE
:102B3F00E0122CC222122B04122AF990101F05A2A8
:102B4F009000097B071204B1122D0E22122B0412D2
:102B5F002AF990103405A29000097B071204B19056
:102B6F000F8205A29000107B0C1204B1900FB605D6
:102B7F00A290001C7B011204B1122D3E900FB705DD
:102B8F00A290001F7B011204B122122B04122AF90A
:102B9F0090103B05A29000097B071204B1122D493A
:102BAF0022122B04122AF990102605A29000097BFD
:102BBF00071204B1900FC805A29000107B101204E9
:102BCF00B190018A122C81122D6A22122B04122A23
:102BDF00F990102605A29000097B071204B1900FFF
:102BEF00D805A29000107B101204B1122DB5122D32
:102BFF00EB22122B04122AF990102D05A290000936
:102C0F007B071204B1900FE805A29000107B101201
:102C1F0004B1900202122C81900232123B85122CC9
:102C2F00E822122B04122AF990102D05A290000908
:102C3F007B071204B1900FF805A29000107B1012C1
:102C4F0004B190021A122C8190024A123B85122C69
:102C5F00E822123B85E075F00C84FEE5F012355B3F
:102C6F0005A29000117B021204B1EE900013120620
:102C7F00D922123B85E09000121206DD90001174EC
:102C8F002BF022900142123B85E01475F006A490C0
:102C9F002CA27390113E022CB7901143022CB790C7
:102CAF001148022CB790114D05A29000167B04120B
:0E2CBF0004B122E0B42B03022CD850FB90008D
:102CCD001D1206DD90001C7450F022C3942A900052
:102CDD001D1206DD90001C7455F022E0B43703027E
:102CED002CFE50FB90001D1206DD90001C7450F060
:102CFD0022C3943690001D1206DD90001C7455F011
:102D0D0022900172123B85E01475F006A4902D1EE1
:102D1D0073901072022D33901082022D3390109209
:102D2D00022D339010A205A29000107B101204B159
:102D3D002290027AE090001D1206DD2290027BE0C7
:102D4D001475F006A4902D56739010D2022D5F903D
:102D5D0010E205A29000107B101204B122900172B6
:102D6D00123B85E0B4010E9010B205A29000167BC7
:102D7D00051204B122B4020D9010B705A2900016F1
:102D8D007B051204B122900172123B85E0B4010A59
:102D9D0090015A123B85122CC222B4020A9001A254
:102DAD00123B85E0122CE8229001D2123B85E014F3
:102DBD0075F006A4902DC5739010BC022DE09010F7
:102DCD00C0022DE09010C4022DE09010C8022DE03D
:102DDD009010CC05A29000147B041204B122900136
:102DED00EA123B85E0B4010E9010D005A290001DB3
:102DFD007B021204B12290001D1206DD22900119F2
:102E0D00E0B40107122EB4122ED022B40207122EF6
:102E1D00EC122F0522B40307122F1E122F3722B4E6
:102E2D000407122F50122F6922B40907122F821294
:102E3D002F9522B40A07122FA8122FBB22900172D0
:102E4D00123B85E0B40304122E882250FA122E5E36
:102E5D0022900119E0B40507122FCE122FEA22B4E9
:102E6D00060412300622B4070712308212309B225C
:102E7D00B408071230B41230CC2222900119E0B4FC
:102E8D0005071230E412310022B4060712311C126C
:102E9D00313522B4070712314E12316A22B40806B9
:102EAD0012318612319F222002012290012A123BFB
:102EBD0085E004120E4DF090012A122C6112322879
:102ECD00C202222003012290012A123B85E0141236
:102EDD000E4DF090012A122C61123228C2032220CD
:102EED00020122900142123B85E004120D1FF012E7
:102EFD002C92123228C2022220030122900142128A
:102F0D003B85E014120D1FF0122C92123228C203D1
:102F1D00222002012290015A123B85E004120D5825
:102F2D00F0122CC2123228C202222003012290017B
:102F3D005A123B85E014120D58F0122CC212322891
:102F4D00C2032220020122900172123B85E004127D
:102F5D000D7EF0122D0E123228C202222003012204
:102F6D00900172123B85E014120D7EF0122D0E129F
:102F7D003228C203222002012290027AE004120EAE
:102F8D005DF0122D3EC202222003012290027AE052
:102F9D0014120E5DF0122D3EC2032220020122906A
:102FAD00027BE004120E70F0122D49C202222003A2
:102FBD00012290027BE014120E70F0122D49C20313
:102FCD00222002012290018A123B85E004120E4D4F
:102FDD00F090018A122C81123228C20222200301A4
:102FED002290018A123B85E014120E4DF090018A59
:102FFD00122C81123228C20322900172123B85E0FD
:10300D00B4010712301E12303722123050123069BF
:10301D00222002012290015A123B85E004120D5824
:10302D00F0122CC2123228C202222003012290017A
:0E303D005A123B85E014120D58F0122CC212EC
:10304B003228C20322200201229001A2123B85E00A
:10305B0004120D6BF0122CE8123228C2022220034C
:10306B0001229001A2123B85E014120D6BF0122C81
:10307B00E8123228C20322200201229001D2123B15
:10308B0085E004120D91F0122DB5123228C20222E6
:10309B00200301229001D2123B85E014120D91F016
:1030AB00122DB5123228C20322200201229001EA0E
:1030BB00123B85E004120DA4F0F546122DEBC20273
:1030CB0022200301229001EA123B85E014120DA489
:1030DB00F0F546122DEBC2032220020122900202D0
:1030EB00123B85E004120E4DF0900202122C81125D
:1030FB003228C2022220030122900202123B85E0F9
:10310B0014120E4DF0900202122C81123228C203BF
:10311B002220020122900232123B85E004120D6B39
:10312B00F0122CE8123228C2022220030122900254
:10313B0032123B85E014120D6BF0122CE812322880
:10314B00C203222002012290021A123B85E00412D4
:10315B000E4DF090021A122C81123228C20222203C
:10316B0003012290021A123B85E014120E4DF090CF
:10317B00021A122C81123228C20322200201229041
:10318B00024A123B85E004120D6BF0122CE812324E
:10319B0028C202222003012290024A123B85E0142E
:1031AB00120D6BF0122CE8123228C2032290027B14
:1031BB00E0B401041231C7221231FC221209EE12C3
:1031CB000A1EB55D0122533DBFF55D120E969001AF
:1031DB001AF0123228900117E0B4010412202522B4
:1031EB00B4020412246722B40406122AF912291C11
:1031FB00221209EE1209B6B43703023210500653ED
:10320B003DBFC20D22433D40200D11D20D90011A3E
:10321B00E004120EB190011AF01231DD22D20A90A5
:10322B00012A123B85E075F00C8485F04E75F00C8D
:10323B00A4F55590015A123B85E0900120F09001C6
:10324B0042123B85E0900124F0121FA61221A3121B
:10325B0037D890018A123B85E0F556900202123B5B
:10326B0085E0F55790021A123B85E0F558900172F4
:10327B00123B85E0900122F01232C7B403041232E4
:10328B00AB2250FA123293222033030232AA90015E
:10329B00A2123B85E0900121F01223E81237F422B1
:1032AB00900232123B85E0900121F01223E8123795
:1032BB00F490024A123B85E012240A22900122E08C
:1032CB00B40103C23322B40202D23322900122E0B2
:1032DB00B4030412331422B404031232E922120A87
:1032EB00121209B6B43703023302500BD294533C7B
:1032FB00FE533DFEC20922C294433C01433D0130C3
:10330B00090122D20912331422120A06120A1E12C2
:10331B000E44B55A1012335A22F55A85575990005C
:10332B003D12333E2250F2F55A85585990004A12FD
:10333B00333E2275F00C8485F06975F00CA4FAE02D
:10334B00F9A3E0C3954EB5690302335AD9F322B5FD
:10335B004D04200A0122C20AF54D254E2A25591289
:10336B0024E2900122E0B40307C294433D01D2361C
:10337B0022E53E20E1012212339512346FE54E1205
:10338B0034921234FEC202C20322E53E20E00574E1
:10339B000002340020E205740102340020E30574BE
:1033AB0002023400E53F20E505740602340020E0FC
:0E33BB0005740302340020E10574040234009E
:1033C90020E305740502340020E205740702340085
:1033D90020E605740802340020E705740902340068
:1033E900E53E20E405740A02340020E505740B0269
:1033F9003400E54EC22E22202E2ED22E854E4FF5B8
:103409004E12343212343E900125E54EF0A3F0F904
:1034190090012A123B85E075F00C8475F00CA42507
:103429004EF012252A1232282290003874041234E0
:10343900491237D82290003DE012345C1237F42249
:10344900FA700122A3E0FC254EC3954F120E26F017
:10345900DAF222FA700122A3E0FC254EC3954F123D
:103469000E26F0DAF2221209FA120A1EB43C0302FD
:10347900347E400122F553B5540122F55475F00C00
:1034890084F55C85F05BD20A22533C21533D4112FD
:103499000E1675F007A49034A373533D41433C02C3
:1034A90022533D41433C0422533D41433C082253AE
:1034B9003D41433C1022533D41433C4022533D4151
:1034C900433C8022533C21433D0222533C21433D4E
:1034D9000422533C21433D0822533C21433D102201
:1034E900533C21433D2022533C21433D8022533C00
:1034F90021533D4122900F8205A290000A7B0412BC
:1035090004B1E54E12355B05A290000E7B02120450
:10351900B190115205A29000107B0A1204B1900FCC
:103529008205A290001A7B031204B1E55490001E93
:103539001206DD90001D742BF022E55B12355B0548
:10354900A290001D7B021204B1E55C90001F1206D7
:10355900D92275F004A49035637390124C2290120D
:103569004E229012502290125222901254229012FE
:1035790056229012582290125A2290125C229012CE
:103589005E229012602290126222900117E0B4012B
:10359900030235AAB402030235AAB404030235AA08
:1035A90022E53E30E10122E53E30E40AE53F30E61E
:1035B90016C212C2132220120DD212E56304120E92
:1035C90034F5631235E12220130DD213E563141289
:1035D9000E34F5631235E122900117E0B4010412AB
:1035E900202522B4020312246722E53E20E10122AC
:1035F90012361E12363212364612365A12366E12EA
:1036090036821236961236AA1236BE1236D21236C1
:10361900E61236FA22E53E30E003C20F22200F08F7
:10362900D20F90005712370E22E53E30E203C21640
:1036390022201608D21690005812370E22E53E3085
:10364900E303C21722201708D21790005912370E28
:1036590022E53F30E003C21822201808D218900052
:103669005A12370E22E53F30E103C2192220190808
:10367900D21990005B12370E22E53F30E303C21ADC
:1036890022201A08D21A90005C12370E22E53F3028
:10369900E503C21B22201B08D21B90005D12370EC6
:1036A90022E53F30E203C21C22201C08D21C9000F4
:1036B9005E12370E22E53F30E603C21D22201D08A7
:1036C900D21D90005F12370E22E53F30E703C21E7C
:1036D90022201E08D21E90006012370E22E53E30CD
:1036E900E403C21F22201F08D21F90006112370E67
:1036F90022E53E30E503C22022202008D220900096
:103709006212370E2205A2900117E0B4010905A241
:10371900123B4212372F22B4020B05A2123B66124A
:103729003B4212377E22E020E01DE560B4040F051C
:0E373900A27B049000561237CD05A20237493C
:1037470050EFE0D2E0F0023753C2E0F07C007B009C
:103757007A3090005705A290003905A2E030E008C2
:103767000BEC05A2F0A305A2A30CDAF0900038EB4E
:10377700F0F56012202522E020E01DE561B40C0F72
:1037870005A27B0C9000861237CD05A20237985010
:10379700EFE0D2E0F00237A2C2E0F07C007B007AD3
:1037A7003090008705A290003E05A2E030E0080BAC
:1037B700EC05A2F0A305A2A30CDAF090003DEBF014
:1037C700F56112246722A3E030E0FBDBF9C2E0F0E9
:1037D70022123810900038E0FBA3E004FA05A2900B
:1037E7000056A3DAFD7401F005A2DBED2212381CA6
:1037F70090003DE0FBA3E004FA05A2900086A3DA5F
:10380700FD7401F005A2DBED2290005774007930BA
:10381700F0A3D9FC2290008774007930F0A3D9FC7B
:103827002212383812390712395D12387212399953
:1038370022E53E20E10122E53F30E60AE53E30E49D
:1038470014C214C2152220140BD21490011CE014C8
:10385700120ECCF02220150BD21590011CE0041299
:103867000ECCF02290000E1206DD2290011CE0B46F
:10387700010122B402071238951238A822B40307AF
:103887001238BB1238CE221238E11238F422200245
:10389700012290011DE004120D0CF012386BC202D8
:1038A700222003012290011DE014120D0CF01238A2
:1038B7006BC203222002012290011EE004120D0CAC
:1038C700F012386BC202222003012290011EE0147D
:1038D700120D0CF012386BC2032220020122900154
:1038E70029E004120EDFF0123951C202222003012F
:1038F70022900129E014120EDFF0123951C203227F
:1039070090011CE0B4010E9011B305A29000057B55
:103917000B1204B122B4020E9011BE12398E90011F
:103927001DE012386B22B4030E9011C912398E9024
:10393700011EE012386B229011D412398E123951C0
:1039470090000E7420F012395122900129E01424BE
:103957004190000FF022900035E06001229011DFC6
:1039670005A29000107B101204B1229011EF05A25E
:103977009000107B101204B122900F7205A29000E4
:10398700107B101204B12205A29000057B091204D6
:10399700B122E53E30E003C20B22200B1BD20B12F3
:1039A70039801201FDC2AF1239C0D2AF12036012C3
:1039B70039729000357404F02290011CE0B40104C0
:1039C700123CF222B40204123D1822B40304123D41
:1039D7002B22123FBA123CF2221239EA123A1D1276
:1039E7003A7122E53E20E10122E53F30E60AE53E55
:1039F70030E414C214C2152220140BD21490011FF4
:103A0700E014120E83F02220150BD21590011FE04F
:103A170004120E83F02290011FE0B401119011FFF0
:103A270005A29000067B0A1204B1123AA622901250
:103A37000905A29000067B0A1204B1123A462290A9
:103A47000128E0B4010E90121305A29000107B101C
:103A57001204B1221414244190001FF09012230580
:103A6700A29000107B0F1204B12290011FE0B40155
:103A770007123A86123A9622123B22123B32222032
:103A8700020122900118E004120CE6F0C202222083
:103A9700030122900118E014120CE6F0C2032290F1
:103AA700123305A29000107B0D1204B1900118E0AB
:0E3AB700B401109010F205A290001D7B0312C6
:103AC50004B1C20C22141490001E1206D9901240A3
:103AD50005A290001D7B011204B190124205A2902F
:103AE500001F7B011204B1D20C22900118E01414BE
:103AF50075F00CA4F565120BB3120AF3E565120B0C
:103B0500B3120AFCE565120BB3120B05E565120B42
:103B1500B3120B0EE565120BB3120B17222002012F
:103B250022900128E004120CF9F0C20222200301C0
:103B350022900128E014120CF9F0C20322E5637506
:103B4500F00CA48582328583337534007535007891
:103B550032F5367537007936120223868208868358
:103B65002285823285833375340075350078327548
:103B7500363075370079361202238682088683220D
:103B8500858232858333753400753500783290012E
:103B95001AE014F536753700793612022386820845
:103BA500868322C3E5829401F582E5839400F5833B
:103BB50022E58229F582E5833400F5832285823268
:103BC500858333753400753500783290011DE01416
:103BD50075F005A4023BF385823285833375340085
:103BE500753500783290011EE01475F00DA4F53698
:103BF50075370079361202238682088683228582EC
:103C050032858333753400753500783275F00502D9
:103C15003C288582328583337534007535007832CA
:103C250075F00DA4F53675370079361202238682B4
:103C35000886832275325575330175340075350054
:103C4500783214F536753700793612023E868208C9
:103C5500868322901C1405A29000007E1005A27F89
:103C650005123C88901C1405A2DEF22290003D0549
:103C7500A29000A07E1005A2790D123CBF90003DD8
:103C8500DEF62274009343D20205A2F0A375D25248
:103C950075D2A2E5D220E0FB53D2FD05A2A3DFE356
:103CA5002290003D05A2901C197B0DE493A305A26B
:103CB500F0A305A2DBF5123C7122E0A343D2020575
:103CC500A2F0A375D25275D2A2E5D220E0FB53D261
:103CD500FD05A2D9E52243D202438E20E0A353D2AB
:103CE500FD538EDF05A2F0A305A2D9EA22790A9039
:103CF500012005A290024005A2123CBF2290012599
:103D0500E54EF0A3E54FF022900125E0F54EA3E046
:103D1500F54F2290003805A2900000123BC205A283
:103D25007905123CBF2290003D05A29000A0123BF0
:103D3500DC05A2790D123CBF22C2AF790A90024080
:103D450005A290012005A2123CDB123D0DD2AF2247
:103D5500C2AF900000C3942B123C0305A290027FD2
:103D650005A27905123CDBD2AF22C2AF9000A0C3F9
:103D75009437123C1705A290003D05A2790D123C1F
:103D8500DBD2AF22C2AF9000A0C39437123C170517
:103D9500A290004A05A2790D123CDBD2AF22E53E86
:103DA50030E10122753C10900F5205A29000007B76
:103DB500101204B1900F6205A29000107B1012043E
:103DC500B1E53E30E1FBE53F30E00630E632023D4D
:103DD500CBE53F30E0FB1201FD1201FD900F7205AE
:103DE500A29000107B101204B11201FD1201FDC258
:103DF500AF123C58123CA6123E11123E51D2AF22D0
:103E0500E53F30E6FB1201FD1201FD229001207411
:103E150016F09001217401F09001227401F09001D7
:103E2500237401F09001247401F09001257400F0D1
:0E3E35009001267400F09001277401F09001B6
:103E4300287401F09001297401F0123CF2229002CF
:103E53007A7418F090027B7401F090012A740012B6
:103E63003EE590018A7400123EE59002027400124E
:103E73003EE590021A7400123EE59001427401126D
:103E83003EE590015A741B123EE5900172740112D3
:103E93003EE59001A2742F123EE59001BA741B1205
:103EA3003EE59001D27403123EE59001EA740112DB
:103EB3003EE59002327401123EE590024A7401120B
:103EC3003EE5123EC9227401900129F0123C3912D9
:103ED3003FC5900129E004F0B40DF174019001296C
:103EE300F0227B18F0A3DBFC22123F8C74A0F912A2
:103EF3003F59123FA2E566F9123F59123FA2E56707
:103F0300F9123F59123FA2123F8C74A1F9123F5983
:103F1300123FA2123F4C123FA8123F7E22E9FA122F
:103F23003F8C74A0F9123F59123FA8E566F9123F7E
:103F330059123FA8E567F9123F59123FA8EAF9124F
:103F43003F59123FA8123F7E22D2A57808123FAEF6
:103F5300E933F9D8F8227808E93392A5F9123FAE8C
:103F6300D8F6227B80DB02800E123F8C74A0F912FC
:103F73003F59123FA840EE123F7E22C2A500D2A4B1
:103F8300000000000000D2A522D2A500D2A40000A8
:103F930000000000C2A5000000000000C2A422C26D
:103FA300A5123FAE22D2A5123FAE220000D2A4003A
:103FB3000000A2A5C2A422900129E0123C39123FBD
:103FC300C52205A290012A05A27FD8123FD77F7D83
:103FD300123FD72285836685826705A2E0F9A30590
:103FE300A2123F20123F66A3DFEA22900129E012CA
:103FF3003C3912401322900128E0B40107900129B3
:10400300E002400C14900129F0123C3912401322B3
:1040130005A290012A05A27FD81240257F7D124078
:104023002522858366858267123EECA3E905A2F00B
:10403300A305A2DFED2275402875410475427D7505
:10404300430275440A90FF9C8582CA8583CB85828F
:10405300CC8583CD43C804D2ADD2AF22C0E0C0D05B
:10406300E582C0E0E583C0E0D2D4C2D3C2CFD5405D
:1040730046754028120306120900120911B20E12E6
:10408300094F30360DD5440A754405D294533DFE8D
:10409300C236D54122754106120988120BFB120C58
:1040A30030D54213754232900035E0600214F0D5EA
:1040B3004305754314B205D0E0F583D0E0F582D013
:0440C300D0D0E03247
:00000001FF
